:040000000C946400F8
:040038000C94BA006A
:14008C00000000000154657374696E67204D41565249432D72
:1400A000494920426F6172642066726F6D2042444D4943520D
:1300B4004F207777772E62646D6963726F2E636F6D0D00DD
:1400C800CFEFD0E1CDBFDEBFC051D0400AEA08830024EBE3FA
:1400DC00F1E011E0ED33F10711F00192FBCF0083ECE8F0E0B1
:1400F000A0E0B1E010E0E73CF10721F0C89531960D92F9CF44
:140104000E943701FFCF8FEF8BBB22242ABA8EEF88BB81E030
:1401180087BB8FEF85BB24BA82BB21BA83B922B88093620052
:14012C00209261008FE18093650020926400089522242EBCE1
:1401400081EC8DBD80E88CBD8EE38BBD80E88ABD8EE389BD24
:1401540080E888BD8EE38093790080E8809378008EE387BD45
:1401680080E886BD2FBC81E08EBD08950A921A922A923A92D4
:14017C004A925A928A93EA930FB60A920E946A0181EC8DBDE8
:1401900080E88CBD40E050E060E070E0409002015090030113
:1401A4002090000130900101241635064606570689F041E01C
:1401B80050E060E070E0241A350A460A570A309201012092CF
:1401CC000001509203014092020103C081E0809304010E9485
:1401E000500109900FBEE991899159904990399029901990D3
:1401F400099018950E944B01F894FE01208031804280538052
:140208003092010120920001509203014092020122242092B8
:14021C0004017894209004012220E1F32496089522242AB873
:140230002BB886E08093950087E689B92092900088E18AB92C
:140244000895F89422242CBE20926D005CDF74DFEBDF222490
:1402580025BE20926A002ABE29BE84E087BF20927D007894DF
:14026C000895EBDF05E011E00E9485010CC0C09A0AEF10E00A
:1402800020E030E0B9DFC0980EEE12E020E030E0B3DFF3CF18
:1402940008953A932A931A930A930895E2E00C9457015A93A1
:1402A8004A930895E1E049915991E0FD089569917991E1FDE7
:1402BC000895A990B990E2FD0895C990D990E3FD0895E990DB
:1402D000F99008957A936A930C9453010E945301402F2090E1
:1402E4003B0130903C01222011F4332021F04A3011F40DE0B6
:1402F800F1DF5D9BFECF4CB9042F11270E94560108950E94B5
:14030C006A01602F712F4427552709C0E62FF72F00810E9435
:140320006E014F5F5F4F6F5F7F4FE62FF72F2080222091F7BD
:100334000AE00E946E0101E010E00E94500108955D
:00000001FF
